:020000040800F2
:1000000000060020A1020008C110000841100008ED
:1000100099100008411000086D100008A3020008A4
:10002000A3020008A3020008A3020008AD2A0008EA
:10003000A3020008A3020008A3020008A30200080C
:10004000A3020008A3020008A3020008A3020008FC
:10005000A3020008A3020008353F0008613F000822
:100060008D3F0008B93F0008E53F0008A3020008E3
:10007000A3020008A3020008A3020008A3020008CC
:10008000A3020008A3020008A3020008A3020008BC
:10009000A3020008A3020008A30200081140000800
:1000A000A3020008A3020008A3020008A30200089C
:1000B000A3020008A3020008A3020008A30200088C
:1000C000A3020008A3020008A3020008A30200087C
:1000D000A3020008A3020008E9400008FD40000850
:1000E00075400008A3020008A3020008A30200084C
:1000F000A3020008A3020008A3020008A30200084C
:10010000A3020008A302000825410008A30200087A
:10011000A3020008A3020008A3020008A30200082B
:10012000A3020008A3020008A3020008A30200081B
:10013000A3020008A3020008A3020008A30200080B
:10014000A3020008A3020008A3020008A3020008FB
:10015000A3020008A3020008A3020008A3020008EB
:10016000A3020008A3020008A3020008A3020008DB
:10017000A302000819360008A3020008A302000821
:10018000A3020008A302000811410008A30200080E
:10019000A3020008A3020008A3020008A3020008AB
:1001A000A3020008A3020008A3020008A30200089B
:1001B000A3020008A3020008A3020008A30200088B
:1001C000A3020008A3020008A3020008A30200087B
:1001D000A302000805360008A3020008A3020008D5
:1001E000A3020008A3020008A3020008A30200085B
:1001F000A3020008A3020008A3020008A30200084B
:10020000A3020008A3020008A3020008A30200083A
:10021000A3020008A3020008A3020008A30200082A
:10022000A3020008A3020008A3020008A30200081A
:10023000A3020008A3020008A3020008A30200080A
:10024000A3020008A3020008A3020008A3020008FA
:10025000A3020008A3020008A3020008A3020008EA
:10026000A3020008A3020008A3020008A3020008DA
:10027000A3020008A3020008A3020008A3020008CA
:10028000A3020008A3020008A3020008A3020008BA
:10029000A3020008A3020008A3020008A3020008AA
:1002A00002E000F000F8FEE772B63A4880F30888F2
:1002B000394880F3098839484EF60851CEF20001DA
:1002C000086040F20000CCF200004EF63471CEF22D
:1002D00000010860BFF34F8FBFF36F8F40F2000043
:1002E000C0F2F0004EF68851CEF200010860BFF374
:1002F0004F8FBFF36F8F4FF00000E1EE100A4EF604
:100300003C71CEF200010860062080F31488BFF330
:100310006F8F02F089FC02F02BFC03F0C5FB4FF05D
:1003200055301F491B4A91423CBF41F8040BFAE784
:100330001C49194A91423CBF41F8040BFAE71A499B
:100340001A4A1B4B9A423EBF51F8040B42F8040B69
:10035000F8E700201749184A91423CBF41F8040BC6
:10036000FAE702F043FC03F023FC144C144DAC42BA
:1003700003DA54F8041B8847F9E700F041F8114C00
:10038000114DAC4203DA54F8041B8847F9E702F038
:100390002BBC000000060020002200200000000806
:1003A0000000002000060020584500080022002020
:1003B0005C22002060220020D44F0020A002000810
:1003C000A0020008A0020008A00200082DE9F04FDA
:1003D0002DED108AC1F80CD0D0F80CD0BDEC108AED
:1003E000BDE8F08F002383F311882846A047002042
:1003F00001F03CFFFEE701F0B7FE00DFFEE7000082
:1004000038B502F03BFB30B1164B00220E211A72B8
:100410005A729972DA7202F007FB054602F03CFB51
:100420000446D0B9104B9D4219D001339D4241F290
:10043000883512BF044600250124002002F0FEFA90
:100440000CB100F079F800F09BFD00F02BFC284681
:1004500000F020F900F070F8F9E70025EDE7054617
:10046000EBE700BF00220020010007B008B500F054
:10047000E5FBA0F120035842584108BD07B541F201
:100480001203022101A8ADF8043000F0F5FB03B01F
:100490005DF804FB38B5202383F311881748C3683F
:1004A0000BB101F069FF0023154A4FF47A7113482C
:1004B00001F026FF002383F31188124C236813B147
:1004C0002368013B2360636813B16368013B636089
:1004D0000D4D2B7833B963687BB9022000F0C0FC66
:1004E000322363602B78032B07D163682BB902207A
:1004F00000F0B6FC4FF47A73636038BD60220020D0
:10050000950400087C23002074220020084B1870FA
:1005100003280CD8DFE800F008050208022000F0EC
:100520008FBC022000F07ABC024B00225A60704758
:10053000742200207C230020F8B5504B504A1C4602
:100540001968013100F0998004339342F8D1626850
:100550004C4B9A4240F291804B4B9B6803F10063F5
:1005600003F500339A4280F08880002000F0B4FB4D
:100570000220FFF7CBFF454B0021D3F8E820C3F85A
:10058000E810D3F81021C3F81011D3F81021D3F8D4
:10059000EC20C3F8EC10D3F81421C3F81411D3F8ED
:1005A0001421D3F8F020C3F8F010D3F81821C3F8C1
:1005B0001811D3F81821D3F8802042F00062C3F854
:1005C0008020D3F8802022F00062C3F88020D3F886
:1005D0008020D3F8802042F00072C3F88020D3F846
:1005E000802022F00072C3F88020D3F8803072B6E9
:1005F0004FF0E023C3F8084DD4E90004BFF34F8F58
:10060000BFF36F8F224AC2F88410BFF34F8F536934
:1006100023F480335361BFF34F8FD2F8803043F619
:10062000E076C3F3C905C3F34E335B0103EA060C5E
:1006300029464CEA81770139C2F87472F9D2203B1D
:1006400013F1200FF2D1BFF34F8FBFF36F8FBFF3C2
:100650004F8FBFF36F8F536923F40033536100232F
:10066000C2F85032BFF34F8FBFF36F8F202383F355
:100670001188854680F308882047F8BD00000208ED
:1006800020000208FFFF0108002200200044025859
:1006900000ED00E02DE9F04F93B0B44B2022FF2194
:1006A00000900AA89D6800F015FCB14A1378A3B920
:1006B0000121B0481170C360202383F31188C368FF
:1006C0000BB101F059FE0023AB4A4FF47A71A948EF
:1006D00001F016FE002383F31188009B13B1A74B92
:1006E000009A1A60A64A1378032B03D000231370D4
:1006F000A24A53604FF0000A009CD3465646D146AA
:10070000012000F09DFB24B19C4B1B68002B00F0E6
:100710002682002000F092FA0390039B002BF2DB6C
:10072000012000F07BFB039B213B1F2BE8D801A29B
:1007300052F823F0B5070008DD070008710800082B
:100740000107000801070008010700080309000865
:10075000D30A0008ED0900084F0A0008770A0008CC
:100760009D0A000801070008AF0A000801070008F9
:10077000210B00085508000801070008650B000858
:10078000C107000855080008010700084F0A0008C3
:100790000107000801070008010700080107000819
:1007A0000107000801070008010700080107000809
:1007B000710800080220FFF759FE002840F0F98177
:1007C000009B022105A8BAF1000F08BF1C4641F2A8
:1007D0001233ADF8143000F04FFA91E74FF47A700D
:1007E00000F02CFA071EEBDB0220FFF73FFE00288B
:1007F000E6D0013F052F00F2DE81DFE807F0030AB3
:100800000D1013360523042105A8059300F034FAD2
:1008100017E004215548F9E704215A48F6E7042176
:100820005948F3E74FF01C08404608F1040800F06F
:1008300055FA0421059005A800F01EFAB8F12C0F16
:10084000F2D101204FF0000900FA07F747EA0B0B3D
:100850005FFA8BFB00F08AFB26B10BF00B030B2B2E
:1008600008BF0024FFF70AFE4AE704214748CDE706
:10087000002EA5D00BF00B030B2BA1D10220FFF70C
:10088000F5FD074600289BD00120002600F024FA41
:100890000220FFF73BFE5FFA86F8404600F02CFA94
:1008A0000446B0B1039940460136A1F140025142DD
:1008B000514100F031FA0028EDD1BA46044641F228
:1008C0001213022105A83E46ADF8143000F0D4F909
:1008D00016E725460120FFF719FE244B9B68AB4223
:1008E00007D9284600F0FAF9013040F06781043555
:1008F000F3E70025224BBA463E461D701F4B5D6054
:10090000A8E7002E3FF45CAF0BF00B030B2B7FF43A
:1009100057AF0220FFF7FAFD322000F08FF9B0F157
:100920000008FFF64DAF18F003077FF449AF0F4AF8
:1009300008EB0503926893423FF642AFB8F5807F1B
:100940003FF73EAF124BB845019323DD4FF47A7069
:1009500000F074F90390039A002AFFF631AF039A6E
:100960000137019B03F8012BEDE700BF00220020B7
:100970007823002060220020950400087C230020BA
:100980007422002004220020082200200C220020D3
:1009900078220020C820FFF769FD074600283FF4B1
:1009A0000FAF1F2D11D8C5F120020AAB25F00300AF
:1009B00084494245184428BF4246019200F064FA37
:1009C000019AFF217F4800F085FA4FEAA803C8F397
:1009D00087027C492846019300F084FA06460028E5
:1009E0003FF46DAF019B05EB830533E70220FFF772
:1009F0003DFD00283FF4E4AE00F0ACF900283FF4E0
:100A0000DFAE0027B846704B9B68BB4218D91F2F3A
:100A100011D80A9B01330ED027F0030312AA134406
:100A200053F8203C05934046042205A9043700F002
:100A300049FB8046E7E7384600F050F90590F2E7B9
:100A4000CDF81480042105A800F016F902E7002370
:100A5000642104A8049300F005F900287FF4B0AEE7
:100A60000220FFF703FD00283FF4AAAE049800F02F
:100A700067F90590E6E70023642104A8049300F0D9
:100A8000F1F800287FF49CAE0220FFF7EFFC00286D
:100A90003FF496AE049800F055F9EAE70220FFF71C
:100AA000E5FC00283FF48CAE00F064F9E1E7022099
:100AB000FFF7DCFC00283FF483AE05A9142000F00A
:100AC0005FF907460421049004A800F0D5F83946E0
:100AD000B9E7322000F0B2F8071EFFF671AEBB078F
:100AE0007FF46EAE384A07EB0903926893423FF6F3
:100AF00067AE0220FFF7BAFC00283FF461AE27F092
:100B000003074F44B9453FF4A5AE484609F104092F
:100B100000F0E4F80421059005A800F0ADF8F1E735
:100B20004FF47A70FFF7A2FC00283FF449AE00F0C2
:100B300011F9002844D00A9B01330BD008220AA9DE
:100B4000002000F0CFF900283AD02022FF210AA887
:100B500000F0C0F9FFF792FC1C4801F08DFB13B0C8
:100B6000BDE8F08F002E3FF42BAE0BF00B030B2BE8
:100B70007FF426AE0023642105A8059300F072F8E7
:100B8000074600287FF41CAE0220FFF76FFC80466A
:100B900000283FF415AEFFF771FC41F2883001F0F8
:100BA0006BFB059800F02CFA46463C4600F0DEF957
:100BB000A6E506464EE64FF0000901E6BA467EE697
:100BC00037467CE67822002000220020A086010023
:100BD0002DE9F84F4FF47A7306460D46002402FBC8
:100BE00003F7DFF85080DFF8509098F900305FFA93
:100BF00084FA5A1C01D0A34210D159F824002A4685
:100C000031460368D3F820B03B46D847854205D12A
:100C1000074B012083F800A0BDE8F88F0134042CB5
:100C2000E3D14FF4FA7001F027FB0020F4E700BF96
:100C3000C82300201022002028420008002307B506
:100C4000024601210DF107008DF80730FFF7C0FFC4
:100C500020B19DF8070003B05DF804FB4FF0FF30B2
:100C6000F9E700000A46042108B5FFF7B1FF80F05C
:100C70000100C0B2404208BD074B0A4630B41978A3
:100C8000064B53F82140014623682046DD69044B9A
:100C9000AC4630BC604700BFC82300202842000893
:100CA000A086010070B50A4E00240A4D01F094FDA3
:100CB000308028683388834208D901F089FD2B6889
:100CC00004440133B4F5003F2B60F2D370BD00BF84
:100CD000CA2300208423002001F05CBE00F10060E4
:100CE00000F500300068704700F10060920000F5E8
:100CF000003001F0D3BD0000054B1A68054B1B887E
:100D00009B1A834202D9104401F062BD0020704753
:100D100084230020CA23002038B50446074D29B19A
:100D200028682044BDE8384001F06ABD28682044A6
:100D300001F054FD0028F3D038BD00BF842300200B
:100D40000020704700F1FF5000F58F10D0F8000828
:100D500070470000064991F8243033B1002308227F
:100D6000086A81F82430FFF7BFBF0120704700BF39
:100D700088230020014B1868704700BF0010005CFA
:100D8000244BF0B51A680446234BC2F30B06120C31
:100D90001F885868BE4293F9085028D09F89BE42E8
:100DA00006D101200C2505FB0033586893F9085043
:100DB00041F201039A421CD041F203039A421AD035
:100DC00042F201039A4218D042F203039A4208BF4A
:100DD0005625621E0B46441E0A4493420FD214F954
:100DE000016F581C6EB1034600F8016CF5E7002056
:100DF000D8E75A25EDE75925EBE75825E9E71846E6
:100E000005E02C2482421C7001D9981C5D70401AA8
:100E1000F0BD00BF0010005C14220020022804D1A5
:100E2000054B4FF080529A6170470128FCD1034B6B
:100E30004FF40022F7E700BF0010025800040258E8
:100E4000022804D1044B4FF480529A617047012864
:100E5000FCD1024B0822F8E70010025800040258A7
:100E6000022805D1064A536983F4805353617047C1
:100E70000128FCD1034A536983F00803F6E700BF59
:100E80000010025800040258002310B5934203D00A
:100E9000CC5CC4540133F9E710BD0000013810B533
:100EA00010F9013F3BB191F900409C4203D11AB1C6
:100EB0000131013AF4E71AB191F90020981A10BDF6
:100EC0001046FCE703460246D01A12F9011B00291E
:100ED000FAD1704702440346934202D003F8011B43
:100EE000FAE770472DE9F8431F4D14460746884638
:100EF00095F8242052BBDFF870909CB395F824300D
:100F00002BB92022FF2148462F62FFF7E3FF95F817
:100F100024004146C0F1080205EB8000A24228BF30
:100F20002246D6B29200FFF7AFFF95F82430A41BFB
:100F300017441E449044E4B2F6B2082E85F82460AB
:100F4000DBD1FFF707FF0028D7D108E02B6A03EBBE
:100F500082038342CFD0FFF7FDFE0028CBD10020D3
:100F6000BDE8F8830120FBE788230020024B1A78B4
:100F7000024B1A70704700BFC823002010220020C7
:100F8000F8B5194C194800F079FC2146174800F0D3
:100F9000A1FC24681648D4F89020164ED2F80438E4
:100FA000154D43F00203114FC2F8043801F064F903
:100FB0002046124900F09CFDD4F890200424D2F879
:100FC000043823F00203C2F804384FF4E1333360ED
:100FD00055F8040BB84202D0314600F0ADFB013C9D
:100FE00014F0FF04F4D1F8BD3C430008C8320020DF
:100FF00040420F00B023002028420008444300086C
:1010000038B50B4B04461A780A4B53F822500A4B5A
:101010009D420CD0094B002118221846FFF75AFFB9
:10102000046001462846BDE8384000F085BB38BD65
:10103000C823002028420008C8320020B023002026
:1010400000B59BB0EFF3098168226846FFF71CFFEB
:10105000EFF30583044B9A6BDA6A9A6A9A6A9A6A82
:101060009A6A9A6A9B6AFEE700ED00E000B59BB0C1
:10107000EFF3098168226846FFF706FFEFF3058367
:10108000044B9A6B9A6A9A6A9A6A9A6A9A6A9B6AF3
:10109000FEE700BF00ED00E000B59BB0EFF3098173
:1010A00068226846FFF7F0FEEFF30583034B5A6BA7
:1010B0009A6A9A6A9A6A9A6A9B6AFEE700ED00E069
:1010C000FEE7000030B50A44084D91420DD011F8FA
:1010D000013B5840082340F30004013B2C4013F02F
:1010E000FF0384EA5000F6D1EFE730BD2083B8ED6E
:1010F000026843681143016003B11847704700005C
:10110000024A136843F0C003136070470044004074
:10111000024A136843F0C003136070470048004060
:10112000024A136843F0C003136070470078004020
:1011300037B5274C274D204600F0F2FA04F1140091
:10114000009400234FF40072234900F0B3F94FF4E8
:101150000072224904F138000094214B00F02CFA6F
:10116000204BC4E91735204C204600F0D9FA04F191
:101170001400009400234FF400721C4900F09AF907
:101180004FF400721A4904F138000094194B00F032
:1011900013FA194BC4E91735184C204600F0C0FA71
:1011A00004F1140000234FF400721549009400F07C
:1011B00081F9144B4FF40072134904F13800009484
:1011C00000F0FAF9114BC4E9173503B030BD00BF88
:1011D000CC23002000E1F50510250020102B002075
:1011E000011100080044004038240020102700208E
:1011F000102D00201111000800480040A4240020F8
:101200001029002021110008102F00200078004034
:10121000037C30B5334C002918BF0C46012B18D184
:10122000314B98420FD1314BD3F8E82042F40032D1
:10123000C3F8E820D3F8102142F40032C3F810219B
:10124000D3F8103105E02A4B98422FD0294B984211
:1012500038D02268036EC16D03EB52038466B3FB82
:10126000F2F36268150442BF23F0070503F0070399
:1012700043EA4503CB60A36843F040034B60E36857
:1012800043F001038B6042F4967343F001030B605B
:101290004FF0FF330B62510505D512F010221DD01F
:1012A000B2F1805F1CD080F8643030BD0F4BD3F8B2
:1012B000E82042F48022C3F8E820D3F8102142F459
:1012C0008022BBE7094BD3F8E82042F08042C3F804
:1012D000E820D3F8102142F08042AFE77F23E2E715
:1012E0003F23E0E738420008CC23002000440258A6
:1012F00038240020A42400202DE9F047C66D0546BF
:101300003768F4692107346219D014F0080118BF56
:101310008021E20748BF41F02001A3074FF02003DE
:1013200048BF41F04001600748BF41F4807183F33A
:101330001188281DFFF7DCFE002383F31188E205E6
:101340000AD5202383F311884FF40071281DFFF77D
:10135000CFFE002383F311884FF020094FF0000ADD
:1013600014F0200838D13B0616D54FF0200905F1BE
:10137000380A200610D589F31188504600F050F93C
:10138000002836DA0821281DFFF7B2FE27F0800377
:101390003360002383F31188790614D5620612D5D1
:1013A000202383F31188D5E913239A4208D12B6CAB
:1013B00033B127F040071021281DFFF799FE376051
:1013C000002383F31188E30618D5AA6E1369ABB125
:1013D0005069BDE8F047184789F31188736A2846B9
:1013E00095F86410194000F0B5F98AF31188F46992
:1013F000B6E7B06288F31188F469BAE7BDE8F08710
:10140000F8B51546826804460B46AA4200D28568A4
:10141000A1692669761AB5420BD218462A46FFF70B
:1014200033FDA3692B44A3612846A3685B1BA3601B
:10143000F8BD0CD9AF1B18463246FFF725FD3A46DA
:10144000E1683044FFF720FDE3683B44EBE71846D2
:101450002A46FFF719FDE368E5E700008368934239
:10146000F7B50446154600D28568D4E90460361AFB
:10147000B5420BD22A46FFF707FD63692B4463612F
:101480002846A3685B1BA36003B0F0BD0DD93246AC
:10149000AF1B0191FFF7F8FC01993A46E06831442F
:1014A000FFF7F2FCE3683B44E9E72A46FFF7ECFC70
:1014B000E368E4E710B50A440024C361029B84603A
:1014C000C16002610362C0E90000C0E9051110BDFE
:1014D00008B5D0E90532934201D1826882B98268A9
:1014E000013282605A1C426119700021D0E9043235
:1014F0009A4224BFC368436100F0DAFE002008BDB1
:101500004FF0FF30FBE7000070B5202304460E4685
:1015100083F31188A568A5B1A368A269013BA36004
:10152000531CA36115782269934224BFE368A36129
:10153000E3690BB120469847002383F311882846BE
:1015400007E03146204600F0A3FE0028E2DA85F3EA
:10155000118870BD2DE9F74F04460E461746984690
:10156000D0F81C904FF0200A8AF311884FF0000B3E
:10157000154665B12A4631462046FFF741FF03462E
:1015800060B94146204600F083FE0028F1D00023D8
:1015900083F31188781B03B0BDE8F08FB9F1000F19
:1015A00003D001902046C847019B8BF31188ED1AA8
:1015B0001E448AF31188DCE7C160C361009B82602E
:1015C0000362C0E905111144C0E9000001617047E0
:1015D000F8B504460D461646202383F31188A76804
:1015E000A7B1A368013BA36063695A1C62611D70C7
:1015F000D4E904329A4224BFE3686361E3690BB122
:1016000020469847002080F3118807E031462046A5
:1016100000F03EFE0028E2DA87F31188F8BD0000F2
:10162000D0E9052310B59A4201D182687AB982685F
:101630000021013282605A1C82611C7803699A423F
:1016400024BFC368836100F033FE204610BD4FF015
:10165000FF30FBE72DE9F74F04460E461746984644
:10166000D0F81C904FF0200A8AF311884FF0000B3D
:10167000154665B12A4631462046FFF7EFFE034680
:1016800060B94146204600F003FE0028F1D0002357
:1016900083F31188781B03B0BDE8F08FB9F1000F18
:1016A00003D001902046C847019B8BF31188ED1AA7
:1016B0001E448AF31188DCE7026843681143016025
:1016C00003B11847704700001430FFF743BF000014
:1016D0004FF0FF331430FFF73DBF00003830FFF705
:1016E000B9BF00004FF0FF333830FFF7B3BF000041
:1016F0001430FFF709BF00004FF0FF311430FFF73F
:1017000003BF00003830FFF763BF00004FF0FF3227
:101710003830FFF75DBF000000207047FFF708BDBD
:10172000044B036000234360C0E9023301230374C8
:10173000704700BF5042000810B52023044683F3D1
:101740001188FFF765FD02232374002383F31188BA
:1017500010BD000038B5C36904460D461BB904210D
:101760000844FFF7A9FF294604F11400FFF7B0FE73
:10177000002806DA201D4FF48061BDE83840FFF7ED
:101780009BBF38BD026843681143016003B118472D
:101790007047000013B5406B00F58054D4F8A438AE
:1017A0001A681178042914D1017C022911D1197900
:1017B000012312898B4013420BD101A94C3002F056
:1017C00073F8D4F8A4480246019B2179206800F000
:1017D000DFF902B010BD0000143001F0F5BF0000C9
:1017E0004FF0FF33143001F0EFBF00004C3002F037
:1017F000C7B800004FF0FF334C3002F0C1B8000012
:10180000143001F0C3BF00004FF0FF31143001F07D
:10181000BDBF00004C3002F093B800004FF0FF3223
:101820004C3002F08DB800000020704710B500F574
:101830008054D4F8A4381A681178042917D1017C8F
:10184000022914D15979012352898B4013420ED1B8
:10185000143001F055FF024648B1D4F8A4484FF4C3
:10186000407361792068BDE8104000F07FB910BD79
:10187000406BFFF7DBBF0000704700007FB5124BE5
:1018800001250426044603600023057400F1840248
:1018900043602946C0E902330C4B02901430019397
:1018A0004FF44073009601F007FF094B04F6944291
:1018B000294604F14C000294CDE900634FF44073D3
:1018C00001F0CEFF04B070BD784200087118000826
:1018D000951700080A68202383F311880B790B33CE
:1018E00042F823004B79133342F823008B7913B16C
:1018F0000B3342F8230000F58053C3F8A4180223E9
:101900000374002383F311887047000038B5037F08
:10191000044613B190F85430ABB90125201D0221C3
:10192000FFF730FF04F114006FF00101257700F09C
:10193000CBFC04F14C0084F854506FF00101BDE879
:10194000384000F0C1BC38BD10B501210446043058
:10195000FFF718FF0023237784F8543010BD0000F0
:1019600038B504460025143001F0BEFE04F14C00E9
:10197000257701F08DFF201D84F854500121FFF7D9
:1019800001FF2046BDE83840FFF750BF90F8803097
:1019900003F06003202B06D190F881200023212A38
:1019A00003D81F2A06D800207047222AFBD1C0E99D
:1019B0001D3303E0034A426707228267C3670120A1
:1019C000704700BF2C22002037B500F58055D5F8B0
:1019D000A4381A68117804291AD1017C022917D178
:1019E0001979012312898B40134211D100F14C0463
:1019F000204602F00DF858B101A9204601F054FF2D
:101A0000D5F8A4480246019B2179206800F0C0F86F
:101A100003B030BD01F10B03F0B550F8236085B081
:101A200004460D46FEB1202383F3118804EB85079D
:101A3000301D0821FFF7A6FEFB6806F14C005B692C
:101A40001B681BB1019001F03DFF019803A901F053
:101A50002BFF024648B1039B2946204600F098F828
:101A6000002383F3118805B0F0BDFB685A69126842
:101A7000002AF5D01B8A013B1340F1D104F180020A
:101A8000EAE70000133138B550F82140ECB12023CB
:101A900083F3118804F58053D3F8A428136852798E
:101AA00003EB8203DB689B695D6845B10421601824
:101AB000FFF768FE294604F1140001F02BFE2046D2
:101AC000FFF7B4FE002383F3118838BD7047000090
:101AD00001F01EB901234022002110B5044600F890
:101AE000303BFFF7F7F90023C4E9013310BD0000D4
:101AF00010B52023044683F311882422416000217D
:101B00000C30FFF7E7F9204601F024F90223237097
:101B1000002383F3118810BD70B500EB81030546E7
:101B200050690E461446DA6018B110220021FFF702
:101B3000D1F9A06918B110220021FFF7CBF9314685
:101B40002846BDE8704001F017BA000083682022E3
:101B5000002103F0011310B5044683601030FFF735
:101B6000B9F92046BDE8104001F092BAF0B4012561
:101B700000EB810447898D40E4683D43A4694581B9
:101B800023600023A2606360F0BC01F0AFBA0000E4
:101B9000F0B4012500EB810407898D40E4683D43E2
:101BA0006469058123600023A2606360F0BC01F0DA
:101BB00025BB000070B502230025044624220370D3
:101BC0002946C0F888500C3040F8045CFFF782F9D1
:101BD000204684F8705001F063F963681B6823B1F4
:101BE00029462046BDE87040184770BD037880F84C
:101BF0008C300523037043681B6810B504460BB195
:101C0000042198470023A36010BD000090F88C20A9
:101C1000436802701B680BB105211847704700002C
:101C200070B590F87030044613B1002380F870301E
:101C300004F18002204601F04FFA63689B68B3B953
:101C400094F8803013F0600535D00021204601F073
:101C5000F9FC0021204601F0E9FC63681B6813B120
:101C6000062120469847062384F8703070BD204630
:101C700098470028E4D0B4F88630A26F9A4288BF13
:101C8000A36794F98030A56F002B4FF0200380F2FA
:101C90000381002D00F0F280092284F8702083F384
:101CA000118800212046D4E91D23FFF771FF00238E
:101CB00083F31188DAE794F8812003F07F0343EA85
:101CC000022340F20232934200F0C58021D8B3F5DE
:101CD000807F48D00DD8012B3FD0022B00F093809D
:101CE000002BB2D104F1880262670222A267E36787
:101CF000C1E7B3F5817F00F09B80B3F5407FA4D1AD
:101D000094F88230012BA0D1B4F8883043F002035C
:101D100032E0B3F5006F4DD017D8B3F5A06F31D0D6
:101D2000A3F5C063012B90D86368204694F8822005
:101D30005E6894F88310B4F88430B047002884D0EB
:101D4000436863670368A3671AE0B3F5106F36D082
:101D500040F6024293427FF478AF5C4B6367022304
:101D6000A3670023C3E794F88230012B7FF46DAFA3
:101D7000B4F8883023F00203A4F88830C4E91D5574
:101D8000E56778E7B4F88030B3F5A06F0ED194F82A
:101D90008230204684F88A3001F0E0F863681B68DE
:101DA00013B1012120469847032323700023C4E97F
:101DB0001D339CE704F18B0363670123C3E723789A
:101DC000042B10D1202383F311882046FFF7BEFE99
:101DD00085F311880321636884F88B5021701B6898
:101DE0000BB12046984794F88230002BDED084F85F
:101DF0008B300423237063681B68002BD6D002212C
:101E000020469847D2E794F8843020461D0603F018
:101E10000F010AD501F052F9012804D002287FF4FD
:101E200014AF2B4B9AE72B4B98E701F039F9F3E706
:101E300094F88230002B7FF408AF94F8843013F0CC
:101E40000F01B3D01A06204602D501F013FCADE70E
:101E500001F004FCAAE794F88230002B7FF4F5AE81
:101E600094F8843013F00F01A0D01B06204602D551
:101E700001F0E8FB9AE701F0D9FB97E7142284F818
:101E8000702083F311882B462A4629462046FFF707
:101E90006DFE85F31188E9E65DB1152284F87020A6
:101EA00083F3118800212046D4E91D23FFF75EFE4D
:101EB000FDE60B2284F8702083F311882B462A4616
:101EC00029462046FFF764FEE3E700BFA84200086A
:101ED000A0420008A442000838B590F870300446CB
:101EE000002B3ED0063BDAB20F2A34D80F2B32D863
:101EF000DFE803F03731310822323131313131310D
:101F000031313737856FB0F886309D4214D2C368BF
:101F10001B8AB5FBF3F203FB12556DB9202383F343
:101F200011882B462A462946FFF732FE85F3118891
:101F30000A2384F870300EE0142384F870302023D4
:101F400083F31188002320461A461946FFF70EFE38
:101F5000002383F3118838BDC36F03B19847002372
:101F6000E7E70021204601F06DFB0021204601F04B
:101F70005DFB63681B6813B1062120469847062362
:101F8000D7E7000010B590F870300446142B29D024
:101F900017D8062B05D001D81BB110BD093B022B69
:101FA000FBD80021204601F04DFB0021204601F026
:101FB0003DFB63681B6813B1062120469847062342
:101FC00019E0152BE9D10B2380F87030202383F31F
:101FD000118800231A461946FFF7DAFD002383F320
:101FE0001188DAE7C3689B695B68002BD5D1C36FA2
:101FF00003B19847002384F87030CEE7024B0022EB
:10200000C3E900339A6070471031002000238268D2
:102010000374054B1B6899689142FBD25A680360B0
:1020200042601060586070471031002008B52023CE
:1020300083F31188037C032B05D0042B0DD02BB91F
:1020400083F3118808BD436900221A604FF0FF3303
:102050004361FFF7DBFF0023F2E7D0E900321360B2
:102060005A60F3E7002382680374054B1B68996884
:102070009142FBD85A680360426010605860704714
:1020800010310020054B1969087418680268536004
:102090001A60186101230374FEF798B9103100200B
:1020A0004B1C30B5044687B00A4D10D02B6901A8EF
:1020B000094A00F025F92046FFF7E4FF049B13B11D
:1020C00001A800F059F92B69586907B030BDFFF736
:1020D000D9FFF8E7103100202D20000838B50C4D4D
:1020E000044641612B6981689A68914203D8BDE832
:1020F0003840FFF78BBF1846FFF7B4FF01232C6170
:10210000014623742046BDE83840FEF75FB900BFA2
:1021100010310020044B1A681B6990689B68984234
:1021200094BF0020012070471031002010B5084CEA
:10213000236820691A6854602260012223611A749E
:10214000FFF790FF01462069BDE81040FEF73EB959
:102150001031002008B5FFF7DDFF18B1BDE80840D9
:10216000FFF7E4BF08BD0000FFF7E0BFFEE7000097
:1021700010B50C4CFFF742FF00F0B4F880220A497A
:10218000204600F03BF8012344F8180C037400F0DB
:102190009DFC002383F3118862B60448BDE810401B
:1021A00000F04CB838310020AC420008BC420008B6
:1021B00000F01CB9EFF3118020B9EFF30583202262
:1021C00082F311887047000010B530B9EFF3058431
:1021D000C4F3080414B180F3118810BDFFF7BAFFEF
:1021E00084F31188F9E70000034A516853685B1AC9
:1021F0009842FBD8704700BF001000E082600222C6
:10220000028270478368A3F17C0243F80C2C0269B8
:1022100043F83C2C426943F8382C074A43F81C2CFD
:10222000C268A3F1180043F8102C022203F8082C0E
:10223000002203F8072C7047E503000810B520239F
:1022400083F31188FFF7DEFF00210446FFF746FF06
:10225000002383F31188204610BD0000024B1B6948
:1022600058610F20FFF70EBF10310020202383F3A9
:102270001188FFF7F3BF000008B50146202383F360
:1022800011880820FFF70CFF002383F3118808BD95
:1022900049B1064B42681B6918605A60136043607D
:1022A0000420FFF7FDBE4FF0FF30704710310020D3
:1022B0000368984206D01A68026050601846596157
:1022C000FFF7A4BE7047000038B504460D462068ED
:1022D000844200D138BD036823605C604561FFF72C
:1022E00095FEF4E7054B4FF0FF3103F11402C3E90B
:1022F00005220022C3E90712704700BF10310020F9
:1023000070B51C4E05460C46C0E9032301F0B6FB30
:10231000334653F8142F9A420DD130620A2C2CBF49
:1023200000190A302A60C5E90124C6E90555BDE84F
:10233000704001F08DBB316A431AE31838BF1C4668
:102340009368A34202D9081901F092FB73699A6855
:1023500094420CD85A68AC602B606A6015609A6829
:102360005D60121B9A604FF0FF33F36170BDA41AD9
:102370001B68ECE71031002038B51B4C63699842AC
:102380000DD08168D0E9003213605A600022C2602B
:102390009A680A449A604FF0FF33E36138BD0368DE
:1023A0002246002142F8143F93425A60C16003D193
:1023B000BDE8384001F056BB9A688168256A0A4436
:1023C0009A6001F05BFB6369411B9A688A42E5D918
:1023D000AB181D1A206A092D98BF01F10A02BDE849
:1023E0003840104401F044BB103100202DE9F04189
:1023F000184C002704F11406656901F03FFB236ABD
:10240000AA68C11A8A4215D81344D5F80C802362F1
:10241000D5E9003213605A606369EF60B34201D1BD
:1024200001F020FB87F311882869C047202383F33C
:102430001188E1E76169B14209D013441B1ABDE874
:10244000F0410A2B2CBFC0180A3001F011BBBDE8C7
:10245000F08100BF1031002000207047FEE700002F
:10246000704700004FF0FF307047000002290CD089
:10247000032904D00129074818BF00207047032A08
:1024800005D8054800EBC20070470448704700209B
:10249000704700BFA04300083C22002054430008BE
:1024A00070B59AB005460846144601A900F0C2F876
:1024B00001A8FEF707FD431C0022C6B25B001046D0
:1024C000C5E9003423700323023404F8013C01AB56
:1024D000D1B202348E4201D81AB070BD13F8011B7C
:1024E000013204F8010C04F8021CF1E708B52023BE
:1024F00083F311880348FFF767FA002383F31188F9
:1025000008BD00BFC832002090F8803003F01F02E1
:10251000012A07D190F881200B2A03D10023C0E9BA
:102520001D3315E003F06003202B08D1B0F8843090
:102530002BB990F88120212A03D81F2A04D8FFF74D
:1025400025BA222AEBD0FAE7034A426707228267BC
:10255000C3670120704700BF3322002007B505295B
:1025600017D8DFE801F0191603191920202383F387
:102570001188104A01210190FFF7CEFA019802213B
:102580000D4AFFF7C9FA0D48FFF7EAF9002383F374
:10259000118803B05DF804FB202383F311880748FA
:1025A000FFF7B4F9F2E7202383F311880348FFF71C
:1025B000CBF9EBE7F442000818430008C8320020CA
:1025C00038B50C4D0C4C2A460C4904F10800FFF7B5
:1025D00067FF05F1CA0204F110000949FFF760FF27
:1025E00005F5CA7204F118000649BDE83840FFF746
:1025F00057BF00BFA04B00203C220020D44200085F
:10260000DE420008E942000870B5044608460D465F
:10261000FEF758FCC6B22046013403780BB91846C1
:1026200070BD32462946FEF739FC0028F3D101205F
:10263000F6E700002DE9F84F05460C46FEF742FC90
:102640002D49C6B22846FFF7DFFF08B10436F6B2BF
:102650002A492846FFF7D8FF08B11036F6B2632E94
:102660000DD8DFF89490DFF894A0DFF89C80DFF8B5
:102670009CB0234F2E7846B92670BDE8F88F2946C6
:102680002046BDE8F84F01F0B9BD252E30D1072214
:1026900049462846FEF702FC70B93B6807350B3403
:1026A00044F80B3C7B6844F8073C3B8924F8033C26
:1026B000BB7A04F8013CDDE7082251462846FEF7C4
:1026C000EDFBA8B9A21C0F4B19780232090911F8C9
:1026D000081002F8041C13F8011B01F00F015B4500
:1026E00011F8081002F8031CEED118340835C1E7C0
:1026F000013504F8016BBDE7C0430008E94200085A
:10270000C843000800E8F11FD44300080CE8F11F9B
:10271000BFF34F8F044B1A695107FCD1D3F8102136
:102720005207F8D1704700BF0020005208B50D4B8A
:102730001B78ABB9FFF7ECFF0B4BDA68D10704D578
:102740000A4A5A6002F188325A60D3F80C21D20743
:1027500006D5064AC3F8042102F18832C3F80421E1
:1027600008BD00BFFE4D0020002000522301674538
:1027700008B5114B1B78F3B9104B1A69510703D5F3
:10278000DA6842F04002DA60D3F81021520705D52A
:10279000D3F80C2142F04002C3F80C21FFF7B8FF38
:1027A000064BDA6842F00102DA60D3F80C2142F0FD
:1027B0000102C3F80C2108BDFE4D0020002000528C
:1027C0000F289ABF00F58060400400207047000089
:1027D0004FF4003070470000102070470F2808B5F4
:1027E0000BD8FFF7EDFF00F500330268013204D18A
:1027F00004308342F9D1012008BD0020FCE700002D
:102800000F2870B5054645D8FFF7D4FC224CFFF7DA
:102810007FFF0646FFF78AFF4FF0FF33072D636106
:10282000C4F8143120D82361FFF772FF2B0243F064
:102830002403E360E36843F08003E36023695A07FD
:10284000FCD42846FFF764FF4FF40031FFF7B8FFD0
:1028500000F002F93046FFF78BFFFFF7B5FC284682
:10286000BDE87040FFF7BABFC4F81031FFF750FF62
:10287000A5F108031B0243F02403C4F80C31D4F87B
:102880000C3143F08003C4F80C31D4F810315B07ED
:10289000FBD4D6E7002070BD002000522DE9F84F90
:1028A00040EA020305460C461746D80602D000202F
:1028B000BDE8F88F27F01F07DFF8D4B0FFF736FF29
:1028C0002744BC4203D10120FFF752FFF0E720224A
:1028D0002946204601F082FC10B920352034F0E76B
:1028E0002B4605F120021E68711CE0D104339A4288
:1028F000F9D1FFF75FFC05F17843234AB3F5801F58
:10290000224B28BF9A4603F1040338BF9046A2F138
:10291000080228BF9846A3F108033ABF9146DA4659
:102920009946FFF7F5FEC8F80060A5EB040CD9F84E
:10293000002004F11C0142F00202C9F80020221F0D
:10294000DAF8006016F00506FAD152F8043F8A4220
:102950004CF80230F4D1BFF34F8FFFF7D9FE4FF0A0
:10296000FF32C8F80020D9F8002022F00202C9F88E
:102970000020FFF729FC20222146284601F02EFCEA
:102980000028AAD030469FE71420005210210052A0
:102990001020005210B5084C237828B11BB9FFF75E
:1029A000C5FE0123237010BD002BFCD02070BDE8B4
:1029B0001040FFF7DDBE00BFFE4D00200244074B74
:1029C000D2B210B5904200D110BD441C00B253F8F1
:1029D000200041F8040BE0B2F4E700BF504000587B
:1029E0000E4B30B51C6F240405D41C6F1C671C6F84
:1029F00044F400441C670A4C02442368D2B243F4F6
:102A000080732360074B904200D130BD441C51F8C5
:102A1000045B00B243F82050E0B2F4E700440258EF
:102A2000004802585040005807B5012201A9002073
:102A3000FFF7C4FF019803B05DF804FB13B504462B
:102A4000FFF7F2FFA04205D0012201A90020019466
:102A5000FFF7C6FF02B010BD0144BFF34F8F064B16
:102A6000884204D3BFF34F8FBFF36F8F7047C3F813
:102A70005C022030F4E700BF00ED00E0002070476A
:102A8000034B1A681AB9034AD2F8D0241A60704767
:102A9000004E00200040025808B5FFF7F1FF024B3E
:102AA0001868C0F3806008BD004E0020EFF3098372
:102AB000054968334A6B22F001024A6383F30988AF
:102AC000002383F31188704700EF00E0202080F39B
:102AD000118862B60D4B0E4AD96821F4E0610904F1
:102AE000090C0A430B49DA60D3F8FC2042F08072EB
:102AF000C3F8FC20084AC2F8B01F116841F0010178
:102B000011601022DA7783F82200704700ED00E0B0
:102B10000003FA0555CEACC5001000E0202310B527
:102B200083F311880E4B5B6813F4006314D0F1EE4D
:102B3000103AEFF309844FF08073683CE361094B6E
:102B4000DB6B236684F30988FFF7E4FA10B1064BC8
:102B5000A36110BD054BFBE783F31188F9E700BFC4
:102B600000ED00E000EF00E0F7030008FA030008C2
:102B700070B5BFF34F8FBFF36F8F1A4A0021C2F8B1
:102B80005012BFF34F8FBFF36F8F536943F400337D
:102B90005361BFF34F8FBFF36F8FC2F88410BFF341
:102BA0004F8FD2F8803043F6E074C3F3C900C3F30B
:102BB0004E335B0103EA0406014646EA817501399A
:102BC000C2F86052F9D2203B13F1200FF2D1BFF3CB
:102BD0004F8F536943F480335361BFF34F8FBFF37B
:102BE0006F8F70BD00ED00E0FEE700000A4B0B4860
:102BF0000B4A90420BD30B4BC11EDA1C121A22F067
:102C000003028B4238BF00220021FEF763B953F85C
:102C1000041B40F8041BECE7B4450008D44F002027
:102C2000D44F0020D44F00207047000070B5D0E989
:102C3000244300224FF0FF359E6804EB42135101FC
:102C4000D3F80009002805DAD3F8000940F08040E5
:102C5000C3F80009D3F8000B002805DAD3F8000BFD
:102C600040F08040C3F8000B013263189642C3F86D
:102C70000859C3F8085BE0D24FF00113C4F81C38C0
:102C800070BD000000EB8103D3F80CC02DE9F043C8
:102C9000DCF814204E1CD0F89050D2F800E005EB80
:102CA000063605EB4118506870450AD30122D5F865
:102CB000343802FA01F123EA0101C5F83418BDE8FD
:102CC000F083AEEB0003BCF81040A34228BF2346BC
:102CD000D8F81849A4B2B3EB840FF0D89468A4F1E3
:102CE000040959F8047F3760A4EB09071F44042F37
:102CF000F7D81C44034494605360D4E7890141F041
:102D00002001016103699B06FCD41220FFF76CBA15
:102D100010B50A4C2046FEF7DDFE094BC4F8903092
:102D2000084BC4F89430084C2046FEF7D3FE074BFE
:102D3000C4F89030064BC4F8943010BD044E002007
:102D4000000008400C440008A04E00200000044091
:102D50001844000870B503780546012B5DD1494B36
:102D6000D0F89040984259D1474B0E216520D3F8B6
:102D7000D82042F00062C3F8D820D3F8002142F0F6
:102D80000062C3F80021D3F80021D3F8802042F07C
:102D90000062C3F88020D3F8802022F00062C3F8DC
:102DA0008020D3F8803000F071FC384BE360384B62
:102DB000C4F800380023D5F89060C4F8003EC02362
:102DC00023604FF40413A3633369002BFCDA01235F
:102DD0000C203361FFF708FA3369DB07FCD41220BB
:102DE000FFF702FA3369002BFCDA00262846A660BA
:102DF000FFF71CFF6B68C4F81068DB68C4F8146840
:102E0000C4F81C68002B3AD1224BA3614FF0FF336A
:102E10006361A36843F00103A36070BD1E4B984239
:102E2000C8D1194B0E214D20D3F8D82042F00072A2
:102E3000C3F8D820D3F8002142F00072C3F8002173
:102E4000D3F80021D3F8802042F00072C3F880202C
:102E5000D3F8802022F00072C3F88020D3F88020BD
:102E6000D3F8D82022F08062C3F8D820D3F800210C
:102E700022F08062C3F80021D3F8003193E7074BBA
:102E8000C3E700BF044E0020004402584014004035
:102E900003002002003C30C0A04E0020083C30C09F
:102EA000F8B5D0F89040054600214FF00066204666
:102EB000FFF724FFD5F8941000234FF001128F681C
:102EC0004FF0FF30C4F83438C4F81C2804EB431228
:102ED00001339F42C2F80069C2F8006BC2F80809CA
:102EE000C2F8080BF2D20B68D5F89020C5F89830DC
:102EF000636210231361166916F01006FBD11220CD
:102F0000FFF772F9D4F8003823F4FE63C4F80038F0
:102F1000A36943F4402343F01003A3610923C4F8D9
:102F20001038C4F814380B4BEB604FF0C043C4F8B2
:102F3000103B094BC4F8003BC4F81069C4F80039D1
:102F4000D5F8983003F1100243F48013C5F89820A7
:102F5000A362F8BDE843000840800010D0F890203C
:102F600090F88A10D2F8003823F4FE6343EA011384
:102F7000C2F80038704700002DE9F84300EB8103E8
:102F8000D0F890500C468046DA680FFA81F9480173
:102F9000166806F00306731E022B05EB41134FF073
:102FA000000194BFB604384EC3F8101B4FF0010166
:102FB00004F1100398BF06F1805601FA03F39169FA
:102FC00098BF06F5004600293AD0578A04F1580107
:102FD000374349016F50D5F81C180B430021C5F841
:102FE0001C382B180127C3F81019A7405369611E1C
:102FF0009BB3138A928B9B08012A88BF5343D8F84E
:103000009820981842EA034301F140022146C8F88B
:103010009800284605EB82025360FFF76FFE08EB2D
:103020008900C3681B8A43EA845348341E43640101
:103030002E51D5F81C381F43C5F81C78BDE8F8831D
:1030400005EB4917D7F8001B21F40041C7F8001B16
:10305000D5F81C1821EA0303C0E704F13F030B4A2B
:103060002846214605EB83035A60FFF747FE05EB30
:103070004910D0F8003923F40043C0F80039D5F8DE
:103080001C3823EA0707D7E700800010000400027D
:10309000D0F894201268C0F89820FFF7C7BD000050
:1030A0005831D0F8903049015B5813F4004004D0F7
:1030B00013F4001F0CBF0220012070474831D0F8E4
:1030C000903049015B5813F4004004D013F4001F02
:1030D0000CBF02200120704700EB8101CB68196A08
:1030E0000B6813604B6853607047000000EB81036E
:1030F00030B5DD68AA691368D36019B9402B84BF65
:10310000402313606B8A1468D0F890201C4402EBB3
:103110004110013C09B2B4FBF3F46343033323F0E1
:10312000030343EAC44343F0C043C0F8103B2B6899
:1031300003F00303012B0ED1D2F8083802EB411043
:1031400013F4807FD0F8003B14BF43F0805343F06A
:103150000053C0F8003B02EB4112D2F8003B43F0B1
:103160000443C2F8003B30BD2DE9F041D0F8906037
:1031700005460C4606EB4113D3F8087B3A07C3F823
:10318000087B08D5D6F814381B0704D500EB81035B
:10319000DB685B689847FA071FD5D6F81438DB0759
:1031A0001BD505EB8403D968CCB98B69488A5A686A
:1031B000B2FBF0F600FB16228AB91868DA68904272
:1031C0000DD2121AC3E90024202383F3118821466B
:1031D0002846FFF78BFF84F31188BDE8F0810123B7
:1031E00003FA04F26B8923EA02036B81CB68002B9C
:1031F000F3D021462846BDE8F041184700EB810393
:103200004A0170B5DD68D0F890306C692668E660D8
:1032100056BB1A444FF40020C2F810092A6802F085
:103220000302012A0AB20ED1D3F8080803EB4214B4
:1032300010F4807FD4F8000914BF40F0805040F0B3
:103240000050C4F8000903EB4212D2F8000940F024
:103250000440C2F800090122D3F8340802FA01F14F
:103260000143C3F8341870BD19B9402E84BF402003
:10327000206020681A442E8A8419013CB4FBF6F4BD
:1032800040EAC44040F00050C6E700002DE9F0419C
:10329000D0F8906004460D4606EB4113D3F8087948
:1032A000C3F80879FB071CD5D6F81038DA0718D50B
:1032B00000EB8103D3F80CC0DCF81430D3F800E045
:1032C000DA6896451BD2A2EB0E024FF000081A6096
:1032D000C3F80480202383F31188FFF78FFF88F35E
:1032E00011883B0618D50123D6F83428AB40134289
:1032F00012D029462046BDE8F041FFF7C3BC0123A8
:1033000003FA01F2038923EA02030381DCF808309F
:10331000002BE6D09847E4E7BDE8F0812DE9F84FAF
:10332000D0F8905004466E69AB691E4016F4805880
:103330006E6103D0BDE8F84FFEF73CBC002E12DAF8
:10334000D5F8003E9F0705D0D5F8003E23F00303D3
:10335000C5F8003ED5F80438204623F00103C5F82F
:103360000438FEF753FC300505D52046FFF75EFC18
:103370002046FEF73BFCB1040CD5D5F8083813F015
:10338000060FEB6823F470530CBF43F4105343F45F
:10339000A053EB60320704D56368DB680BB12046AD
:1033A0009847F30200F1BA80B70226D5D4F890907E
:1033B00000274FF0010A09EB4712D2F8003B03F453
:1033C0004023B3F5802F11D1D2F8003B002B0DDA4A
:1033D00062890AFA07F322EA0303638104EB870395
:1033E000DB68DB6813B13946204698470137D4F8CB
:1033F0009430FFB29B689F42DDD9F00619D5D4F80E
:103400009000026AC2F30A1702F00F0302F4F012EE
:10341000B2F5802F00F0CC80B2F5402F09D104EB3B
:103420008303002200F58050DB681B6A974240F05E
:10343000B2803003D5F8185835D5E90303D50021FB
:103440002046FFF791FEAA0303D501212046FFF78E
:103450008BFE6B0303D502212046FFF785FE2F0369
:1034600003D503212046FFF77FFEE80203D50421A0
:103470002046FFF779FEA90203D505212046FFF774
:1034800073FE6A0203D506212046FFF76DFE2B026C
:1034900003D507212046FFF767FEEF0103D508217A
:1034A0002046FFF761FE700340F1A980E90703D5CC
:1034B00000212046FFF7EAFEAA0703D50121204696
:1034C000FFF7E4FE6B0703D502212046FFF7DEFE7F
:1034D0002F0703D503212046FFF7D8FEEE0603D5BC
:1034E00004212046FFF7D2FEA80603D50521204679
:1034F000FFF7CCFE690603D506212046FFF7C6FE7E
:103500002A0603D507212046FFF7C0FEEB0576D536
:1035100020460821BDE8F84FFFF7B8BED4F89090D8
:1035200000274FF0010AD4F894305FFA87FB9B68BC
:103530009B453FF639AF09EB4B13D3F8002902F452
:103540004022B2F5802F24D1D3F80029002A20DAB6
:10355000D3F8002942F09042C3F80029D3F800299B
:10356000002AFBDB5946D4F89000FFF7C7FB2289FD
:103570000AFA0BF322EA0303238104EB8B03DB68D3
:103580009B6813B159462046984759462046FFF795
:1035900079FB0137C7E7910701D1D0F80080072AEE
:1035A00002F101029CBF03F8018B4FEA18283DE7A6
:1035B00004EB830300F58050DA68D2F818C0DCF819
:1035C0000820DCE9001CA1EB0C0C00218F4208D183
:1035D000DB689B699A683A449A605A683A445A6030
:1035E00027E711F0030F01D1D0F800808C4501F1DD
:1035F000010184BF02F8018B4FEA1828E6E7BDE815
:10360000F88F000008B50348FFF788FEBDE80840C2
:10361000FFF784BA044E002008B50348FFF77EFE8A
:10362000BDE80840FFF77ABAA04E0020D0F89030ED
:1036300003EB4111D1F8003B43F40013C1F8003B08
:1036400070470000D0F8903003EB4111D1F80039F9
:1036500043F40013C1F8003970470000D0F89030EF
:1036600003EB4111D1F8003B23F40013C1F8003BF8
:1036700070470000D0F8903003EB4111D1F80039C9
:1036800023F40013C1F8003970470000090100F16C
:103690006043012203F56143C9B283F8001300F0CF
:1036A0001F039A4043099B0003F1604303F5614304
:1036B000C3F880211A60704730B50433039C01724F
:1036C000002104FB0325C160C0E90653049B03638A
:1036D000059BC0E90000C0E90422C0E90842C0E936
:1036E0000A11436330BD00000022416AC260C0E994
:1036F0000411C0E90A226FF00101FEF7E5BD0000E8
:10370000D0E90432934201D1C2680AB9181D70474A
:1037100000207047036919600021C2680132C2604D
:10372000C269134482699342036124BF436A0361FF
:10373000FEF7BEBD38B504460D46E3683BB162698D
:103740000020131D1268A3621344E36207E0237A8A
:1037500033B929462046FEF79BFD0028EDDA38BD37
:103760006FF00100FBE70000C368C269013BC36062
:103770004369134482699342436124BF436A4361AE
:1037800000238362036B03B11847704770B5202391
:10379000044683F31188866A3EB9FFF7CBFF0546DE
:1037A00018B186F31188284670BDA36AE26A13F83F
:1037B000015B9342A36202D32046FFF7D5FF0023AB
:1037C00083F31188EFE700002DE9F84F04460E4619
:1037D000174698464FF0200989F311880025AA461C
:1037E000D4F828B0BBF1000F09D141462046FFF7BD
:1037F000A1FF20B18BF311882846BDE8F88FD4E9EA
:103800000A12A7EB050B521A934528BF9346BBF14A
:10381000400F1BD9334601F1400251F8040B91428D
:1038200043F8040BF9D1A36A403640354033A36214
:10383000D4E90A239A4202D32046FFF795FF8AF380
:103840001188BD42D8D289F31188C9E730465A465B
:10385000FDF71AFBA36A5E445D445B44A362E7E79D
:1038600010B5029C0433017204FB0321C460C0E95B
:1038700006130023C0E90A33039B0363049BC0E9DA
:103880000000C0E90422C0E90842436310BD000003
:10389000026A6FF00101C260426AC0E9042200229C
:1038A000C0E90A22FEF710BDD0E904239A4201D1F3
:1038B000C26822B9184650F8043B0B6070470020DC
:1038C00070470000C3680021C2690133C3604369C7
:1038D000134482699342436124BF436A4361FEF704
:1038E000E7BC000038B504460D46E3683BB12369E8
:1038F00000201A1DA262E2691344E36207E0237A02
:1039000033B929462046FEF7C3FC0028EDDA38BD5E
:103910006FF00100FBE7000003691960C268013A1B
:10392000C260C269134482699342036124BF436A3F
:10393000036100238362036B03B1184770470000E3
:1039400070B520230D460446114683F31188866A1C
:103950002EB9FFF7C7FF10B186F3118870BDA36AB7
:103960001D70A36AE26A01339342A36204D3E16942
:1039700020460439FFF7D0FF002080F31188EDE7DF
:103980002DE9F84F04460D46904699464FF0200A1F
:103990008AF311880026B346A76A4FB949462046E4
:1039A000FFF7A0FF20B187F311883046BDE8F88FFC
:1039B000D4E90A073A1AA8EB0607974228BF174628
:1039C000402F1BD905F1400355F8042B9D4240F8C8
:1039D000042BF9D1A36A40364033A362D4E90A2309
:1039E0009A4204D3E16920460439FFF795FF8BF32F
:1039F00011884645D9D28AF31188CDE729463A463F
:103A0000FDF742FAA36A3D443E443B44A362E5E726
:103A1000D0E904239A4217D1C3689BB1836A8BB162
:103A2000043B9B1A0ED01360C368013BC360C3699B
:103A30001A4483699A42026124BF436A03610023E6
:103A400083620123184670470023FBE700F0DAB8D1
:103A5000034B002258631A610222DA60704700BFEC
:103A6000000C0040014B0022DA607047000C00405F
:103A7000014B5863704700BF000C0040014B586A6F
:103A8000704700BF000C00404B6843608B68836048
:103A9000CB68C3600B6943614B6903628B69436206
:103AA0000B6803607047000008B53C4B40F2FF71A3
:103AB0003B48D3F888200A43C3F88820D3F88820ED
:103AC00022F4FF6222F00702C3F88820D3F888208E
:103AD000D3F8E0200A43C3F8E020D3F808210A43D2
:103AE000C3F808212F4AD3F808311146FFF7CCFF5D
:103AF00000F5806002F11C01FFF7C6FF00F5806051
:103B000002F13801FFF7C0FF00F5806002F15401B7
:103B1000FFF7BAFF00F5806002F17001FFF7B4FF14
:103B200000F5806002F18C01FFF7AEFF00F58060C8
:103B300002F1A801FFF7A8FF00F5806002F1C401BF
:103B4000FFF7A2FF00F5806002F1E001FFF79CFFA4
:103B500000F5806002F1FC01FFF796FF02F58C7121
:103B600000F58060FFF790FF00F000F90E4BD3F8EE
:103B7000902242F00102C3F89022D3F8942242F03E
:103B80000102C3F894220522C3F898204FF0605236
:103B9000C3F89C20054AC3F8A02008BD0044025881
:103BA000000002582444000800ED00E01F00080354
:103BB00008B500F0F3FAFEF7DBFA0F4BD3F8DC2080
:103BC00042F04002C3F8DC20D3F8042122F0400286
:103BD000C3F80421D3F80431084B1A6842F00802F4
:103BE0001A601A6842F004021A60FEF749FFBDE845
:103BF0000840FEF7E5BC00BF004402580018024828
:103C000070470000114BD3F8E82042F00802C3F8D7
:103C1000E820D3F8102142F00802C3F810210C4A22
:103C2000D3F81031D36B43F00803D363C722094B99
:103C30009A624FF0FF32DA6200229A615A63DA60C8
:103C40005A6001225A611A60704700BF004402584E
:103C50000010005C000C0040094A08B51169D368E7
:103C60000B40D9B29B076FEA0101116107D52023F0
:103C700083F31188FEF79CFA002383F3118808BDB3
:103C8000000C0040384B4FF0FF31D3F88020C3F8D0
:103C90008010D3F880200022C3F88020D3F8800061
:103CA000D3F88400C3F88410D3F88400C3F88420C8
:103CB000D3F88400D86F40F0FF4040F4FF0040F498
:103CC0003F5040F03F00D867D86F20F0FF4020F40D
:103CD000FF0020F43F5020F03F00D867D86FD3F8A2
:103CE00088006FEA40506FEA5050C3F88800D3F85C
:103CF0008800C0F30A00C3F88800D3F88800D3F81E
:103D00009000C3F89010D3F89000C3F89020D3F837
:103D10009000D3F89400C3F89410D3F89400C3F83B
:103D20009420D3F89400D3F89800C3F89810D3F8EF
:103D30009800C3F89820D3F89800D3F88C00C3F803
:103D40008C10D3F88C00C3F88C20D3F88C00D3F8F7
:103D50009C00C3F89C10D3F89C10C3F89C20D3F8A7
:103D60009C3000F0E7B900BF00440258614B0122CB
:103D7000C3F80821604BD3F8F42042F00202C3F8E4
:103D8000F420D3F81C2142F00202C3F81C210222C5
:103D9000D3F81C31594BDA605A689104FCD5584A63
:103DA0001A6001229A60574ADA6000221A614FF4C1
:103DB00040429A61514B9A699204FCD51A6842F4C8
:103DC00080721A604C4B1A6F12F4407F04D04FF48B
:103DD00080321A6700221A671A6842F001021A60DC
:103DE000454B1A685007FCD500221A611A6912F077
:103DF0003802FBD1012119604FF0804159605A67A8
:103E0000414ADA62414A1A611A6842F480321A6001
:103E1000394B1A689103FCD51A6842F480521A6033
:103E20001A689204FCD53A4A3A499A6200225A63C7
:103E300019633949DA6399635A64384A1A64384A0B
:103E4000DA621A6842F0A8521A602B4B1A6802F024
:103E50002852B2F1285FF9D148229A614FF4886262
:103E6000DA6140221A622F4ADA644FF080521A65F2
:103E70002D4A5A652D4A9A6532232D4A13601368DC
:103E800003F00F03022BFAD11B4B1A6942F0030215
:103E90001A611A6902F03802182AFAD1D3F8DC2024
:103EA00042F00052C3F8DC20D3F8042142F0005263
:103EB000C3F80421D3F80421D3F8DC2042F0804277
:103EC000C3F8DC20D3F8042142F08042C3F8042177
:103ED000D3F80421D3F8DC2042F00042C3F8DC2000
:103EE000D3F8042142F00042C3F80421D3F804318E
:103EF000704700BF0080005100440258004802583B
:103F000000C000F0020000010000FF0100889008DE
:103F100032206000630209011D0204004704050805
:103F2000FD0BFF01200000200010E0000001010057
:103F3000002000524FF0B04208B5D2F8883003F0AC
:103F40000103C2F8883023B1044A13680BB15068EA
:103F50009847BDE80840FEF7E1BD00BF544F002080
:103F60004FF0B04208B5D2F8883003F00203C2F82F
:103F7000883023B1044A93680BB1D0689847BDE8F4
:103F80000840FEF7CBBD00BF544F00204FF0B042B9
:103F900008B5D2F8883003F00403C2F8883023B1A2
:103FA000044A13690BB150699847BDE80840FEF711
:103FB000B5BD00BF544F00204FF0B04208B5D2F855
:103FC000883003F00803C2F8883023B1044A9369AB
:103FD0000BB1D0699847BDE80840FEF79FBD00BF10
:103FE000544F00204FF0B04208B5D2F8883003F0AB
:103FF0001003C2F8883023B1044A136A0BB1506A27
:104000009847BDE80840FEF789BD00BF544F002027
:104010004FF0B04310B5D3F8884004F47872C3F879
:104020008820A30604D5124A936A0BB1D06A984738
:10403000600604D50E4A136B0BB1506B98472106EE
:1040400004D50B4A936B0BB1D06B9847E20504D5AE
:10405000074A136C0BB1506C9847A30504D5044A6A
:10406000936C0BB1D06C9847BDE81040FEF756BD7D
:10407000544F00204FF0B04310B5D3F8884004F4FB
:104080007C42C3F88820620504D5164A136D0BB133
:10409000506D9847230504D5124A936D0BB1D06D2E
:1040A0009847E00404D50F4A136E0BB1506E984741
:1040B000A10404D50B4A936E0BB1D06E98476204ED
:1040C00004D5084A136F0BB1506F9847230404D5E9
:1040D000044A936F0BB1D06F9847BDE81040FEF7CC
:1040E0001DBD00BF544F002008B50348FDF704F97B
:1040F000BDE80840FEF712BDCC23002008B50348F8
:10410000FDF7FAF8BDE80840FEF708BD38240020A6
:1041100008B50348FDF7F0F8BDE80840FEF7FEBC1F
:10412000A424002008B5FFF797FDBDE80840FEF77E
:10413000F5BC0000062108B50846FFF7A7FA0621DE
:104140000720FFF7A3FA06210820FFF79FFA0621B0
:104150000920FFF79BFA06210A20FFF797FA0621AC
:104160001720FFF793FA06212820FFF78FFA09217D
:104170007A20FFF78BFA07213220FFF787FA0C210C
:104180002620FFF783FA0C212720FFF77FFA0C2166
:104190005220BDE80840FFF779BA000008B5FFF7E4
:1041A00071FD00F00DF8FDF7B9FAFDF791FCFDF790
:1041B00063FBFFF725FDBDE80840FFF747BC0000A3
:1041C0000023054A19460133102BC2E9001102F100
:1041D0000802F8D1704700BF544F002010B50139D4
:1041E0000244904201D1002005E0037811F8014F0C
:1041F000A34201D0181B10BD0130F2E7034611F8AD
:10420000012B03F8012B002AF9D1704753544D3389
:104210003248373F3F3F0053544D333248373433F1
:104220002F37353300000000C8320020CC23002097
:1042300038240020A4240020009600000000000084
:10424000000000000000000000000000000000006E
:1042500000000000E5160008D11600080D17000840
:10426000F916000805170008F1160008DD16000809
:10427000C91600081917000800000000F51700080B
:10428000E11700081D180008091800081518000893
:1042900001180008ED170008D917000829180008B0
:1042A0000000000001000000000000006D61696E68
:1042B0000000000069646C6500000000B442000862
:1042C00050310020C8320020010000006D2100089C
:1042D000000000004172647550696C6F74002542E3
:1042E0004F415244252D424C002553455249414CE3
:1042F000250000000200000000000000151A000860
:10430000851A000840004000704B0020804B0020C0
:104310000200000000000000030000000000000098
:10432000CD1A00080000000010000000904B002093
:10433000000000000100000000000000044E00200A
:10434000010102005D2500086D2400080925000810
:10435000ED240008430000005C430008090243000C
:10436000020100C03209040000010202010005241C
:1043700000100105240100010424020205240600A6
:1043800001070582030800FF09040100020A00007A
:1043900000070501024000000705810240000000FF
:1043A00012000000A84300081201100102000040A2
:1043B000091241570002010203010000040309042D
:1043C00025424F415244250050697850696C6F7402
:1043D0002D56360030313233343536373839414294
:1043E000434445460000000000000000211C000876
:1043F000D91E0008851F0008400040003C4F0020E7
:104400003C4F0020010000004C4F002080000000C5
:10441000400100000800000000010000000400004E
:10442000080000000000802A00000000AAAAAAAA32
:1044300000000024FFFF00000000000000A00A00B0
:104440004000000008000000AAAAAAAA000000007C
:10445000FFFF00000000000000000000100000143A
:1044600000000000AAAAAAAA10000014FFFF000082
:10447000000000000000000010681A0000000000AA
:10448000AAAAAAAA10541500FFFF00000000700796
:10449000770000000081020100100000AAAAAAAA69
:1044A00000410100FFFF0000000000700700000055
:1044B0000000000000000000AAAAAAAA0000000054
:1044C000FFFF0000000000000000000000000000EE
:1044D00000000000AAAAAAAA00000000FFFF000036
:1044E00000000000000000000000000000000000CC
:1044F000AAAAAAAA00000000FFFF00000000000016
:10450000000000000000000000000000AAAAAAAA03
:1045100000000000FFFF000000000000000000009D
:104520000000000000000000AAAAAAAA00000000E3
:10453000FFFF00000000000000000000000000007D
:1045400000000000AAAAAAAA00000000FFFF0000C5
:1045500000000000000000003B040000000000001C
:1045600000001E0000000000FF000000000000002E
:104570000C4200083F0000005004000017420008F1
:104580003F000000009600000000080096000000B8
:104590000008000004000000BC4300080000000008
:1045A000000000000000000000000000000000000B
:0445B0000000000007
:00000001FF
